:030000000219FDE5
:03000B000200AA46
:03002B0002015679
:03005B000202E5B9
:030073000202D2B4
:1000800002030406080C10182030406080040608A3
:100090000C10182030406080A0C00003070F1F0D17
:1000A0000D0403060D0502030202C2AFC0D0C0E07A
:1000B000206214E5256009E473E525F4F58AD2622F
:1000C000D0E0D0D0D2AF3285268AC262E526F46075
:1000D00029D0E0D0D0C292C291C290D2AF32C292A7
:1000E000C291C290206F0C2066097405D5E0FDE531
:1000F0007B4290D0E0D0D0D2AF32758A00C28DD290
:100100006201F301B9306805206602D29201B9306C
:100110006805206602D29101B9306805206602D2D6
:100120009001B9C29530680A2066077446D5E0FD93
:10013000D29201B9C29430680A2066077446D5E0AD
:10014000FDD29101B9C29330680A2066077446D582
:10015000E0FDD29001B9C2AFC2AD53E6EFC0D0C04E
:10016000E0D2D3D2AFC2CEE52A6007207449152A67
:1001700021B77800790020742EE580307E01F430BC
:10018000E70278FF53DACF207E0343DA20307E0384
:1001900043DA10C2D8C271E580307E01F430E70244
:1001A00079FFC3E89970CB306103752A402074034E
:1001B000752A40885CD27020740DE52B6004152BE5
:1001C00021C743DA01C2D820700221DAA85C20617D
:1001D00002C27020740221D888227882B604038576
:1001E0002224C3E52594404002D26420CF0AD0E007
:1001F000D0D043E610D2AD32C2CF053A7802E52A1C
:100200006005307402152AC3E55C94014005755FF2
:10021000004124756000756900E55F2401F55F50B9
:1002200003755FFF7982B7020D306E1DC3E522941E
:10023000324016854C227982B7030E306E0BC3E52F
:100240002294324004798E8722C3E52395226008E8
:100250004004152341580523D8CA0569E569700291
:100260001569D56A63756A017805C3E569956B40C0
:1002700057C3E569956C50087801756A0302028CD2
:10028000C3E569956D50057801756A01C3E562950E
:1002900024401E7982B7040241BD206E1485246279
:1002A000E569046003856B69756A0175233C020288
:1002B000C8E5622850057562FF41BDF562E562043C
:1002C00070067560FF7569FFD0E0D0D043E610D2AC
:1002D000AD32C2AF53E67F7592FA7593FFC2607577
:1002E0009104D2AF32C2AF53E6EFC2ADC0D0C0E08E
:1002F000C0F0D2D3D2AFA8FBA9FCC2D83071026142
:100300004C53DACF207E0343DA10307E0343DA20E9
:10031000D271E580307E01F420E7026123882789CD
:1003200028A13153DACF207E0343DA20307E034305
:10033000DA10C2D8C271307402A11D7800E5803095
:100340007E01F430E702A11D885CA10553DACF20BD
:100350007E0343DA20307E0343DA10C2712061024B
:10036000812553DACF207E0343DA10307E0343DA4F
:1003700020C2D8D27188578958C3E89555F8E995B5
:1003800056F97B007E087A00C3E8948CE99400500B
:1003900005755B008117882178A2E6A8216055C306
:1003A000E894C8E994005008E4D2E4FB7A0A61F2C8
:1003B000C3E89468E994015008E4D2E3FB7A0F6142
:1003C000F2C3E894D0E994025008E4D2E2FB7A1E2A
:1003D00061F2C3E894A0E994055008E4D2E1FB7A05
:1003E0003C61F2C3E89498E994085008E4D2E0FB39
:1003F0007A787E00C3E89559FCE9955AFD30E70A02
:10040000ECF42401FCEDF43400FD755B00C3EC9AC0
:10041000ED9E5003755B018859895A85575585585B
:10042000567802A105C3E89527F8E99528F9307CAC
:100430000281E9307B0281E9307A0281E220750293
:100440008148E9FDE8FC8167E9C313F9E813F83056
:10045000790281E2E9C313F9E813F830780281E206
:10046000E9C313FDE813FC20612CC3EC941CED944C
:0E047000024002817EED701EC3EC94C850184D
:10047E000529E52970021529C3E529940A5002A120
:10048E001D755C00D270A11DE5296002152974004E
:10049E00207F037896E624FAFEE43400FFC3EC9E38
:1004AE00FCED9FFD50067800790081E9C3EC94FFC6
:1004BE00ED9400400678FF790081E9EC8572F0A496
:1004CE00C5F0A2F733F87900400302050578FF79ED
:1004DE0000020505E9C313F9E813F8307C0EE96054
:1004EE000278FFC3E81338F8E43400F9C3E894FF48
:1004FE00E99400400278FF885CD270206102A11D51
:10050E00741FF4552F4BF52FC274EB7002D2747515
:10051E002A40307403752A0A306102A13120740317
:10052E0053DAFE207403752B20D0F0D0E0D0D0D259
:10053E00AD43E61032790102056179030205617956
:10054E000A020561791E020561796402056179C8A6
:10055E000205617817E4D5E0FDD8FAD9F6227A14AF
:10056E007B780205887A107B8C0205887A0D7BB425
:10057E000205887A0B7BC80205887902E4C294D5FD
:10058E00E0FDD291D5E0FDC291D5E0FDD294D5E04B
:10059E00FDE920E002D29230E002D290E573D5E080
:1005AE00FDE920E002C29230E002C2907496D5E0DE
:1005BE00FDD9C9EAF8D5E0FDD8FBDBBEC29422C353
:1005CE007C007D0075F00005F0EA33FAEB33FB504A
:1005DE00F6EB13FBEA13FAC3E9FFE8FEE89AF8E933
:1005EE009BF95004EFF9EEF8B3EC33FCED33FDD587
:1005FE00F0DFEDF9ECF822E889F08A20D2D4F8A9E0
:10060E00F07B0030F70B7BFFF42401F8E9F43400A3
:10061E00F9E88520F0A4ADF0F8E98520F0A4AFF05C
:10062E00FEED2EF974003FFA7C04C3EA13FAE913C7
:10063E00F9E813F8DCF48BF030F70AE8F42401F84B
:10064E00E9F43400F9E889F0C2D4F8A9F0227882EE
:10065E00B604030206FBC3E55C9419401EE52D5457
:10066E00067018206E3678057994E7146007780ABC
:10067E001460027812C3E54198401F306E098564FC
:10068E00627569FF756A01852224E4F544F545F526
:10069E0046F547F548C26E0206FBD26E7994E71412
:1006AE007013E523F43333F913F8E9540104F9E830
:1006BE0054FE0206EFE714147014E523F4333333BB
:1006CE00F913F8E9540304F9E854FC0206F7E5239C
:1006DE00F433333333F913F8E954070404F9E854C7
:1006EE00F8C39440F8E99400F98844894522C3E59B
:1006FE004113F9E54013F8C3E54498F8E54599F937
:10070E00500CC3E89480E994FF4016020733C3E807
:10071E00947FE994005003020733787F7900020733
:10072E0033788079FF8849894A22E5492546F8E5DC
:10073E004A3547F9854A20E4300701F43548FA3046
:10074E00E709C3EA94F04015020771C3EA940F500B
:10075E000302077178FF79FF7A0F0207717800792B
:10076E00007AF0C3E5249561500AC37401952450B4
:10077E000B02078FE54A20E70E02078FE54A30E7A6
:10078E0006884689478A482278A5E6FAC3E54933A2
:10079E00F8E54A33F9D105E930E70BC3E89480E96F
:1007AE0094FF4013E1C9C3E8947FE994005002E13D
:1007BE00C9787F7900E1C9788079FFE820E715C311
:1007CE00E52398F84009C3E8940140030207F07846
:1007DE00010207F0E8F424012523F840030207F094
:1007EE0078FF884B2278A6E6FAA847A948D105E9F2
:1007FE0030E70CC3E89401E994FF4016020824C3C5
:10080E00E894FFE99400500302082478FF7900026F
:10081E000824780179FFE920E715C3E54B98F840E5
:10082E0009C3E89401400302084B780102084BE823
:10083E00F42401254BF8400302084B78FF8824224C
:10084E0078FFC26420693D206A12D264C3E54194E8
:10085E000A4009C3E52594405002C26479A1E760BD
:0E086E0023E541601F74FF8541F0848539F059
:10087C00306A0375F005A4F8C5F0600278FFC3E890
:10088C0095645002A864886322C3E5409440E54116
:10089C009401E56350031401A6046002F563227809
:1008AC0083E6F520120F2375E89012054375E89046
:1008BC00E5E820ECFBA8BDA9BE120FC9756E5575F5
:1008CC006F00C3740013FD7455606613FC74552CD3
:1008DC00FC74003DFDECFAEDFBC3E89AE99B401477
:1008EC00E56E2455F56EE56F3400F56FEA2CFAEBE6
:1008FC003DFB80E5AE6EAF6FC3E56F13F9E56E138C
:10090C00F8C3E913F9E813F87A03C3E913F9E81308
:10091C00F8DAF7AA201A7009756E00756F000209D3
:10092C003D1AEA6008EE28FEEF39FFDAF88E6E8F7A
:10093C006F2275E890227883E6FFE5E820ECF7A8B3
:10094C00BDA9BE0570C3E57094084052757000E9EE
:10095C00FA79A0E76044EA7007E571601B02097838
:10096C00C3E895716010E5715006600C140209849F
:10097C000460F9020984E571F571C3946D401B752F
:10098C0061C0C394044013756180C39404400B751B
:10099C006140C39404400375610075BB0622EFC32C
:1009AC009401601F7455601BC3E894FFE9940350D5
:1009BC0012C3E8956EE9956F5009E561600C1561FD
:1009CC000209D6E561F460020561A861C3E52498CB
:1009DC005002A824C3E89562400AA862E562F4605C
:1009EC000385626188258826E570B4070375BB1002
:1009FC0022743279A787F0A4C5F0A2F733F8C3E8C4
:100A0C0095614002A86188228824882588268864FC
:100A1C00227540007541F022C2AF75C820A8CCA940
:100A2C00CDAA3A30CF010A75C824D2AFAB3BAC3C4F
:100A3C00883B893CC3E89BF8E99C206908F930673E
:100A4C00026130418DAD3D8A3DF9EA9DFA60047832
:100A5C00FF79FFAE3EAF3F8B3E8C3FA83BA93CC31A
:100A6C00E89EF8E99FF9C3E54113FBE54013FAE86A
:100A7C002AF540E93BF54150067540FF7541FF41B1
:100A8C00D7AA40AB41AC40AD417E047F02C3EB948E
:100A9C000440021E1FC3EB940840021E1FC3ED133B
:100AAC00FDEC13FCDEF7C3EA9CFAEB9DFBEF60094F
:100ABC00C3E913F9E813F8DFF7EA28FAEB39FB8AF4
:100ACC00408B4150067BFF8B408B41C3EB94025013
:100ADC0002D2673069047F0361027892E6FFC3E5B6
:100AEC0037948240110FC3E53794A040010FC3EF38
:100AFC00940640027F057E02E541C4540FF9E5419E
:100B0C00C454F0F8E540C4540F28F8C3E89EFAE941
:100B1C009400FB4009C3EA9402EB940050047A025F
:100B2C00E4FB617CAA40AB41EBC4FEEAC4540F4E1B
:100B3C00FCC3EA9CFAEB9400FBC3E813C313F8EA7A
:100B4C0028FAEB3400FB8A408B41C3EB9402400241
:100B5C00C2677802EBC4FE7B00EAC4540F4EFAC3A2
:100B6C00EA98FA4005C3940250027A027892E6FFA2
:100B7C00306002617C855192855293D26043E6804D
:100B8C00C3E49AF8E49BF93067028108E8FAE9FBC0
:100B9C00D3E913FDE813FC88518952C3EF94036029
:100BAC0038EF20E00DE82CF8E93DF9ECFAEDFB020A
:100BBC000BD1E828F8E939F9C3E82402F8E9340044
:100BCC00F97AFE7BFFC3EF9403400E8A538B548853
:100BDC004D894E8C4F8D50813C885389548A4D8B56
:100BEC004E8C4F8D503069127553F07554FF754F04
:100BFC00F07550FF7551F07552FF813CE8FAD3E85F
:100C0C0013FC8851C3EF94036020EF20E007E82C1D
:100C1C00F8ECFA8128E8282402F87AFEC3EF940352
:100C2C0040088A53884D8C4F813C88538A4D8C4F99
:100C3C00E568C3335002646BF56830600281467519
:100C4C003402D26043E680E52D54066034A840A9F6
:100C5C0041C3E913F9E813F8C3E913F9E813F830C1
:0F0C6C006904E92440F9C2AF53E67F759100C3D4
:100C7B00E498F594E499F595759104D26043E68078
:100C8B00D2AF22D265754300752000306C037520FE
:100C9B0040020CADD265754300752040306C037576
:100CAB00200078017901206720E52D54066002C2EF
:100CBB00657914E541C313700104F8C39414400221
:100CCB007814306904781B791B206010E543600CA5
:100CDB00306903D53404D26DA150914E0543E59B89
:100CEB00F45440B52002A13A30690908C3E8994091
:100CFB00011881D420650A08C3E899400281AD81AF
:100D0B00D4C265C2AF53E67F7591003067127594FC
:100D1B00007595FE759104D26043E680D2AF81AD2C
:100D2B00AE40AF41C3E49EF594E49FF595A11FC37C
:100D3B00E5339401500281AD30650281ADD802A13B
:100D4B004E81D4C26DC2AF53E67F7591008553942B
:100D5B00855495759104854D92854E93D26043E6EB
:100D6B0080D2AFE52D54066008206A020533020DD0
:100D7B008C306D0D206C0A206507158115810215CD
:100D8B00FC2278003064053065027801E53775F098
:100D9B0007A4F9E5F028F5F0E9A2F013A2F113A2EC
:100DAB00F213F537C394785003753778C3E537954D
:100DBB00384008D266C292C291C290306002A1C67E
:100DCB00854F92855093D26043E68022207D16C2D8
:100DDB00AF754202C294D295306202D290D2AF75F7
:100DEB009F11020FC6C2AF754202C294D2933062FA
:100DFB0002D292D2AF759F11020FC6307243207D83
:100E0B0020C2AF754203900134757B10C290C29320
:100E1B00306204D291C124D294D2AF759F01020FDC
:100E2B00C6C2AF754203900134757B10C292C29556
:100E3B00306204D291C144D294D2AF759F21020F7C
:100E4B00C6207D17C2AF75420390010FC29030626E
:100E5B0002D291D2AF759F01020FC6C2AF7542038A
:100E6B0090010FC292306202D291D2AF759F2102D4
:100E7B000FC6207D16C2AF754204C295D293306265
:100E8B0002D291D2AF759F21020FC6C2AF75420439
:100E9B00C293D295306202D291D2AF759F01020FED
:100EAB00C6307243207D20C2AF7542059001237579
:100EBB007B20C291C294306204D292C1CAD295D225
:100ECB00AF759F11020FC6C2AF75420590014575F4
:100EDB007B08C291C294306204D290C1EAD293D201
:100EEB00AF759F11020FC6207D17C2AF75420590DB
:100EFB000105C291306202D292D2AF759F11020FDF
:100F0B00C6C2AF754205900119C2913062EBD29007
:100F1B00D2AF759F11020FC6207D16C2AF75420668
:100F2B00C293D294306202D292D2AF759F01020F5C
:100F3B00C6C2AF754206C295D294306202D290D22D
:100F4B00AF759F21020FC6307243207D20C2AF7553
:100F5B004201900145757B08C292C295306204D262
:100F6B0090E170D293D2AF759F21020FC6C2AF75BD
:100F7B004201900123757B20C290C293306204D250
:100F8B0092E190D295D2AF759F01020FC6207D17CB
:100F9B00C2AF754201900119C292306202D290D257
:100FAB00AF759F21020FC6C2AF754201900105C2FA
:100FBB0090306202D292D2AF759F01C2662290012D
:100FCB0003757B00C292C291C290C295C294C29328
:100FDB00C2622278807607087607087601087604C5
:100FEB000876FF0876FF08760B087602087601086C
:100FFB007601788C76010876000876B40876FF08BF
:10100B0076FF0876FF0876030876FF0876010876E8
:10101B00FF0876250876D00876780876C808760417
:10102B000876FF08760108760008767A08760708B6
:10103B0076010876010876000876FF08760022789C
:10104B0087E6FFC2727888C27DE630E102D27DC2AC
:10105B007E7889E630E102D27EC3EF940260087598
:0F106B008E01D273021077758E00C273227880C7
:10107A00E6149000809378A5F67881E614900080B3
:10108A009378A6F67886E61490008D9378A7F6787A
:10109A009FE6F8700108C3E8941140027811E82825
:1010AA0028F56B256B256B28F56C256B2828F56DC3
:1010BA007886E6F539C394025003753902789CE6BE
:1010CA007538FFB402037538A0B403037538827803
:1010DA00A3E61490009A93F566120FC92222789615
:1010EA00E6FA7897E6FB7888E6B40305C3EB940E34
:1010FA00FB307F047A007BFFC3EB9AFCC3948250D7
:10110A00027C827572000572EC8572F0A4C3E5F068
:10111A00947D40F222D27F11E81205527A007B00B8
:10112A007C10120548E55C2AFA74003BFBDCF37C70
:10113A0004C3EB13FBEA13FADCF7FEC27F11E822C1
:10114A00E5EF20E6037520000520903FFFE5201417
:10115A006006901DFF1460009304600375EF10533E
:10116A00D9BF7581C043FF8012054375EF0043B2B2
:10117A0003E5B3240220E70DF521E5E320E0068527
:10118A0021B343E301120FC97580FF75A40075F1FD
:10119A009075D47F75900075A53F75F23F75D5009F
:1011AA0075A60175E241120FC9E4F8F6D8FD756813
:1011BA0001120FDE12165378988673753001C2AF8A
:1011CA0012055C12056C12055212057312055212B1
:1011DA00057A12055212177612055C12055C120581
:1011EA0057C2AF78FA79FA308707D9FBD8F7021CC9
:1011FA0000114A117811E711E878988673120FC91D
:10120A0075881075890275C82475910475D840755A
:10121A00A82275B80275E690759B80759D0075D1F8
:10122A000E75BC5875BB0675BA1175E88012054370
:10123A00D2AF1208AB75360053DACF207E0343DAF9
:10124A0020307E0343DA1043DA01C2D8C271120594
:10125A005CD2617B037A0CE55B70077A0CDB0302D4
:10126A0011EB1205522070030211EBC270E55CC348
:10127A00940240E1E52F541F855E5DF55EB55DD5AC
:10128A00DAD5C26153DACF207E0343DA20307E03F7
:10129A0043DA10C2D8C27178A2E67008D274E52F78
:1012AA0054E0F52FC275752900120557307409C329
:1012BA00E529940A4002D275120548780230740270
:1012CA007800C3E55C9840F0C2AF12056C12056C59
:1012DA0012056CD2AF12055C754C00120548788C69
:1012EA00E6C3940150030213BBE530C394015003D3
:1012FA000213BB207435C3E55C94FF50030213BB91
:10130A00C2AF120581D2AF120557C3E55C940150F2
:10131A00EFC2AF12056C12054D12056CD2AF120561
:10132A0057C3E55C94FF40E90217FB7F05D27F11A2
:10133A00E8120557C2AFC27F11E8AE5CC3E55C9400
:10134A007FD2AF4076120543C2AF120581D2AFDF1A
:10135A00DC311FC3EE94057897F612055C121695D8
:10136A0012177E7F0AD27F11E8120557C2AFC27FD9
:10137A0011E8AE5CC3E55C947FD2AF50E612054338
:10138A00C2AF12056C12054D12056CD2AFDFD63111
:10139A001FEE24037896F612055C1216951217AD05
:1013AA0012055711E8C3E55C94FF500241FD02178C
:1013BA00FBC3E55C954C4003855C4C1205577801EC
:1013CA007988E7B403027805C3E55C98400241E5F1
:1013DA00C2AF120581120581120581D2AF12055CD6
:1013EA00753000E4F531F5320531E531F4703F0529
:1013FA0032789AE67819146012783214600D787D82
:10140A0014600878FA146003753200C3E532984014
:10141A001D120FC91205431532753100789986736A
:10142A00C2AF120581D2AF7898867312055712059A
:10143A004DE52A700530740221EB78012074027898
:10144A0006C3E55C9840A1120557E52A700302110C
:10145A00EBC2AF120FC9E4F522F523F524F525F501
:0F146A0026F567D2AF7885E6C333F565E4F54420
:10147900F545F546F547F548F570F52CF52DF537A1
:1014890075700875BB1012054312093EE5E820EC9A
:10149900FBA8BDA9BEE97001F888711209427570EF
:1014A9000875BB10114AC2AF7561FF1209FD85228B
:1014B90061852262852263D2AF7522017524017587
:1014C9002501752601856069756A017888E6B40386
:1014D90007C27D307602D27DD268D2697533001297
:1014E9000F23120F52120A1D120A24120A1D120A80
:1014F90024120A1D120C9F12065C120D8D120DD7B3
:10150900120A24120C8E306E031206FC2067031295
:10151900084E306703120895120D8D120E06120A35
:1015290024120C9F306E03120738120D8D120E7D96
:10153900120A24120C8E306E03120796120D8D12A8
:101549000EAC120A24120C9F306E031207F3120D0F
:101559008D120F23120A2412093E120C8E120D8DC0
:10156900120F52120942120A2430692C85646185CE
:101579006462856069756A0179187A0CC3E53399E3
:101589004009C269D26A8A350215A1C3E55C940192
:1015990040030214FD021604306A1D206C1AE53559
:1015A900147006C26AD26B81FDF535C3E55C9401FE
:1015B90040030214FD021604753600C3E55F940169
:1015C9004009856462856069756A0178FA79A4E7DA
:1015D90060027803C3E55F985021307404E52A60FE
:1015E9001A78F0306C058564617820C3E54198501C
:1015F9000281FD0536E55C6002C107753600C2AFA0
:10160900120FC97887E6FE7602114A7887EEF6E46A
:10161900F522F523F524F525F526F565752C0075D4
:101629002D00D2AF120557120FC978A4E66006D271
:1016390092D291D290307406E52A700221EB788D0E
:10164900E6C39401400241C261ED901A0D7820125F
:1016590016D7E520B4A50CA31216D7E520B45A0372
:10166900021675120FDE121695021694901A037857
:10167900807B0A1216D7A308DBF9901A0F788C7BA6
:10168900191216D7A308DBF9901A2822C2AF12172C
:10169900161216F0901A00740E1216DCA3740612B4
:1016A90016DCA374151216DC901A0378807B0A12D3
:1016B90016DBA308DBF9901A0F788C7B191216DB5D
:1016C900A308DBF9121729121707901A2822E493A5
:1016D900F622E6438F01538FFD75EF0275B7A575A5
:1016E900B7F1F0538FFE22438F02438F0175EF024A
:1016F90075B7A575B7F1901A0DF0538FFC22901AA2
:101709000D74A5D1DC901A0E745AD1DC227A307985
:10171900D07820901A40D1D7E520F709A3DAF7222B
:101729007A3079D0901A40E7D1DC09A3DAF922ABF3
:1017390074A875BB01027980BB02027981BB0302DF
:101749007982BB04027994BB05027983BB060279CD
:1017590086BB07027992BB08027987BB0902799C8B
:10176900BB0A027988BB0B027989E8F7227C05124A
:10177900055CDCFB22C2AF12056C12057312057AF7
:1017890012058112054D12056C12057312057A12A4
:10179900058112054D12056C12057312057A1205A1
:1017A90081D2AF22C2AF12058112057A12057312D6
:1017B900056C12054D12058112057A120573120581
:1017C9006C12054D12058112057A12057312056C0A
:1017D900D2AF22AE74AF75C2AF12056C12056C128E
:1017E900056C12054DDEF212058112054DDFF8D2A6
:1017F900AF22F17EF1761217767574017575017550
:1018090076001217DC7C05AD5C12055CC3ED955CB6
:1018190070F5C3E55C9401400AC3E55C94FF403769
:1018290002183D12173812169512177EC2AF75EFBE
:1018390010121776DCD10576C3E576940350028041
:10184900C11217760575E5741490009F93F808C3C3
:10185900E57598500280A81217761217760574C399
:0E186900E574940C50028094120FDE12169556
:08187700C2AF75EF10121776E5
:0319FD0002114A8A
:101A00000E061507070104FFFF0B020101A55A018D
:101A100000B4FFFFFF03FF01FF25D078C804FF01DA
:091A200000FF07010100FF00FFB7
:101A400023585031324123202020202020202020E4
:101A500023424C48454C4923463333302320202031
:101A60002020202020202020202020202020202076
:101C0000C2AFC2D353D9BF7581C043B20343FF8073
:101C1000752438752503B1C975EF0275E24043F1AB
:101C20008053A47F75D4FFD2877DFA780379E67C50
:101C300010752200752300901DD67B0675249875BB
:101C400025013087028142208708D8FBD9F9DCF7CB
:101C500081B4308708D8FBD9F9DCF781B4B189E4C5
:101C600093A3C39A6004DDC381B4DBDBB17B600264
:101C7000812B7B08E493FAA3B15CDBF87A30B15C8A
:101C8000752200752300B17BEAFCEBFDC3ED94FEE9
:101C9000400EB17B8A278B28ED30E0048A828B834B
:101CA000B17B7AC270D8C3ED94FE601350CEBD00F4
:101CB00025EC60097520007521FF0200008100A855
:101CC00027A9280809D804D90281D3B17FEA89AAB3
:101CD000F281C50D81A0C3ED94035049EDA2E092BD
:101CE000007AC5C3E5829400E583941C50902000DF
:101CF00010438F02438F0175B7A575B7F1F030001F
:101D00001FA827A9280809438F01538FFDD804D99C
:101D100002A12089AAE275B7A575B7F1F0A3A10DBC
:101D2000538FFC817C7AC1BD030CE493A3FAB140CC
:101D3000DCF8B138817C817EAA22AB23B15CEBFA5E
:101D4000EA6222752608C3E52313F523E52213F57D
:101D50002250066323A0632201D526EAB1C9B1C986
:101D600075260AEAF4200102D287300102C287B147
:101D7000C9C3134002C201D526EB22B17FEAFB2082
:101D80008702A17F308702A184752608AE24AF2583
:101D9000C3EF13FFEE13FEB1CDB1C9C3EA13308711
:101DA000024480FA30E703632201C3E52313F523DD
:101DB000E52213F52250066323A0632201D526D91C
:101DC000E52265236523F52222AE24AF250E0FDE22
:101DD000FEDFFCD20122424C48656C693437316326
:041DE000F3300601D5
:00000001FF
